:100000000C9434000C9451000C9451000C94510049
:100010000C9451000C9451000C9451000C9451001C
:100020000C9451000C9451000C9451000C9451000C
:100030000C9451000C9451000C9451000C945100FC
:100040000C9451000C9451000C9451000C945100EC
:100050000C9451000C9451000C9451000C945100DC
:100060000C9451000C94510011241FBECFEFD8E026
:10007000DEBFCDBF13E0A0E0B1E0E4E1FFE102C0EC
:1000800005900D92A635B107D9F723E0A6E5B3E0B8
:1000900001C01D92A939B207E1F70E94060C0C9429
:1000A000880F0C9400000895E82FF0E0E957FC4F0A
:1000B00080810895E82FF0E0E957FC4F60830895B0
:1000C000E82FF0E0EE0FFF1FE959FC4F808191818E
:1000D0000895E82FF0E0EE0FFF1FE159FC4F8081FB
:1000E00091810895E82FF0E0EE0FFF1FE958FC4FD3
:1000F000808191810895E82FF0E0EE0FFF1FE15815
:10010000FC4F808191810895E82FF0E0EE0FFF1FF2
:10011000E95AFC4F808191810895E82FF0E0EE0FBD
:10012000FF1FE15AFC4F80819181089524B12C6218
:1001300024B92A9A25B1277D25B920E52CBD2A9816
:1001400020EF2EBD0DB407FEFDCF9EBD0DB407FE02
:10015000FDCF8EBD0DB407FEFDCF6EBD0DB407FE05
:10016000FDCF2A9A81E0089524B12C6224B92A9AFD
:1001700025B1277D25B920E52CBD2A982FE02EBD7D
:100180000DB407FEFDCF9EBD0DB407FEFDCF8EBDA5
:100190000DB407FEFDCF1EBC0DB407FEFDCF8EB51E
:1001A0002A9A089524B12C6224B92A9A25B1277D70
:1001B00025B920E52CBDFB019B01240F351F60EF05
:1001C000E217F307A9F02A986EBD0DB407FEFDCF24
:1001D0009EBD0DB407FEFDCF8EBD0DB407FEFDCF55
:1001E00071917EBD0DB407FEFDCF2A9A0196E8CF2E
:1001F000CA01089524B12C6224B92A9A25B1277D19
:1002000025B920E52CBDFB019B01240F351F6FE0B4
:10021000E217F307B1F02A986EBD0DB407FEFDCFCB
:100220009EBD0DB407FEFDCF8EBD0DB407FEFDCF04
:100230001EBC0DB407FEFDCF7EB571932A9A0196C0
:10024000E7CFCA0108952F923F924F925F926F922B
:100250007F928F929F92AF92BF92CF92DF92EF9256
:10026000FF920F931F93CF93DF93CDB7DEB72897FD
:100270000FB6F894DEBF0FBECDBF282E362E86E116
:1002800091E00E94A30C622D8BE190E00E94960009
:10029000632D8AE190E00E94960080E090E49093C4
:1002A000600380935F0380E090E69093580380930F
:1002B000570381E291E00E94A30C87E5882E83E03A
:1002C000982E9FE5A92E93E0B92E2FE633E03887CC
:1002D0002F8307E613E027E7C22E23E0D22E3FE765
:1002E000E32E33E0F32E1A821982412C512C1C820A
:1002F0001B82612C712C222D30E03E832D83232C18
:10030000312CAF81B88511961C921E92F801118292
:1003100010822B813C8121153042B4F58D819E8164
:10032000098002C0959587950A94E2F78370992712
:1003300082309105A9F083309105D9F0019739F009
:1003400080E094E08D939C93EFEFF3E01AC0E0E03F
:10035000F8E0AF81B885ED93FC93EFEFF7E011C0C3
:10036000E0E0F0E1AF81B885ED93FC93EFEFFFE0C3
:1003700008C0E0E0F0E2AF81B885ED93FC93EFEFC9
:10038000FFE1D701ED93FC934114F0E25F069CF589
:10039000C101098002C0959587950A94E2F78370A0
:1003A000992782309105A9F083309105D1F001970A
:1003B00041F0E0E0F4E0D801ED93FC93EFEFF3E0DF
:1003C00017C0E0E0F8E0D801ED93FC93EFEFF7E021
:1003D0000FC0E0E0F0E1D801ED93FC93EFEFFFE018
:1003E00007C0E0E0F0E2D801ED93FC93EFEFFFE10E
:1003F000D601ED93FC93AF81B8858D919D91B8871F
:10040000AF832B813C81280F391F3C832B83D8017C
:100410002D913D918D01420E531E61147104D9F04E
:10042000EF81F885349760817181F50132974081C1
:100430005181460F571FF50151834083FD013497C9
:1004400060817181F401329740815181460F571FBD
:10045000D4014D935C93F40160817181F2E08F0EC1
:10046000911CD5014C9111965C91B2E0AB0EB11C80
:100470003F932F939F938F937F936F935F934F93AC
:100480007F926F92AAE4B1E0BF93AF930E948D0C6C
:10049000FFEF6F1A7F0A29813A812E5F3F4F3A831F
:1004A000298332E0C30ED11C42E0E40EF11C0FB6EA
:1004B000F894DEBF0FBECDBF94E06916710409F059
:1004C00020CF28960FB6F894DEBF0FBECDBFDF91C8
:1004D000CF911F910F91FF90EF90DF90CF90BF9041
:1004E000AF909F908F907F906F905F904F903F90D4
:1004F0002F900895682F80E090E80C94960080E893
:100500000C947A02CF93DF93EC01688181E090E054
:100510000E949600698182E090E00E9496006A81C4
:1005200083E090E00E9496006B8184E090E0DF9190
:10053000CF910C949600CF93DF93EC0181E090E093
:100540000E94B400888382E090E00E94B400898316
:1005500083E090E00E94B4008A8384E090E00E94EF
:10056000B4008B83DF91CF910895CF93DF93EC019B
:10057000688185E090E00E949600698186E090E0C5
:100580000E9496006A8187E090E00E9496006B814D
:1005900088E090E0DF91CF910C949600CF93DF93A9
:1005A000EC01688189E090E00E94960069818AE010
:1005B00090E00E9496006A818BE090E00E94960095
:1005C0006B818CE090E00E9496006C818DE090E061
:1005D0000E9496006D818EE090E0DF91CF910C94A7
:1005E0009600CF93DF93EC0168818FE090E00E944A
:1005F0009600698180E190E00E9496006A8181E125
:1006000090E00E9496006B8182E190E0DF91CF91B3
:100610000C94960085E190E00C94B400CF93C82F21
:10062000692F87E190E00E9496006C2F88E190E0AE
:10063000CF910C949600682F89E190E00C9496007D
:10064000682F86E190E00C949600CF93DF93EC0145
:1006500081E090E00E94B400888382E090E00E94F4
:10066000B400898383E090E00E94B4008A8384E030
:1006700090E00E94B4008B83DF91CF910895CF93D7
:10068000DF93EC0185E090E00E94B400888386E06F
:1006900090E00E94B400898387E090E00E94B4005B
:1006A0008A8388E090E00E94B4008B83DF91CF9131
:1006B0000895CF93DF93EC0189E090E00E94B400AD
:1006C00088838AE090E00E94B40089838BE090E008
:1006D0000E94B4008A838CE090E00E94B4008B8377
:1006E0008DE090E00E94B4008C838EE090E00E9448
:1006F000B4008D83DF91CF910895CF93DF93EC0108
:100700008FE090E00E94B400888380E190E00E9436
:10071000B400898381E190E00E94B4008A8382E181
:1007200090E00E94B4008B83DF91CF9108950F93E6
:100730001F93CF93DF938B01C82FD0E02496DC2F3B
:10074000CC27CE0106960E94B400F8018083CE012A
:1007500007960E94B400F8018183CE0108960E949A
:10076000B400F8018283CE0109960E94B400F8011A
:100770008383CE010A960E94B400F8018483CE01DF
:100780000B960E94B400F8018583DF91CF911F91F1
:100790000F9108950F931F93CF93DF938B01C82F71
:1007A000D0E02496DC2FCC27FB016081CE01069699
:1007B0000E949600F8016181CE0107960E94960082
:1007C000F8016281CE0108960E949600F8016381CB
:1007D000CE0109960E949600F8016481CE010A9626
:1007E0000E949600F8016581CE010B96DF91CF91B2
:1007F0001F910F910C9496000F931F93CF93DF934B
:100800008B01C82FD0E02496DC2FCC27CE010C968C
:100810000E94B400F8018083CE010D960E94B400BE
:10082000F8018183CE010E960E94B400F801828304
:10083000CE010F960E94B400F8018383DF91CF911F
:100840001F910F9108950F931F93CF93DF938B0107
:10085000C82FD0E02496DC2FCC27FB016081CE018D
:100860000C960E949600F8016181CE010D960E94BF
:100870009600F8016281CE010E960E949600F80162
:100880006381CE010F96DF91CF911F910F910C9450
:1008900096000F931F93CF93DF938B01C82FD0E067
:1008A0002496DC2FCC27CE0140960E94B400F8019C
:1008B0008083CE0141960E94B400F8018183DF91CC
:1008C000CF911F910F9108950F931F93CF93DF93B3
:1008D0008B01C82FD0E02496DC2FCC27FB01608150
:1008E000CE0140960E949600F8016181CE014196AA
:1008F000DF91CF911F910F910C9496001F93CF938E
:10090000DF93162F672FC82FD0E02496DC2FCC273B
:10091000CE0142960E949600612FCE014396DF9150
:10092000CF911F910C94960090E0982F88278A5EB3
:100930009B4F0C94960090E0982F88278C5E9B4FDD
:100940000C94960090E0982F88278E5F9B4F0C9414
:10095000B40090E0982F88278D5F9B4F0C94B400D3
:10096000CF92DF92EF92FF920F931F93CF93DF937B
:10097000C82FD0E02496DC2FCC277E0180E2E80E41
:10098000F11CA19600E010E0C7010E94B400C82E3F
:10099000D12CDC2CCC24CE010E94B400C80ED11C7A
:1009A000C114D10461F0C7010E94B400082F10E007
:1009B000102F0027CE010E94B400080F111D0C1546
:1009C0001D0511F7C801DF91CF911F910F91FF9085
:1009D000EF90DF90CF900895CF92DF92EF92FF9249
:1009E0000F931F93CF93DF93C82FD0E02496DC2F73
:1009F000CC277E0186E2E80EF11CA79600E010E00D
:100A0000C7010E94B400C82ED12CDC2CCC24CE010E
:100A10000E94B400C80ED11CC114D10461F0C701FA
:100A20000E94B400082F10E0102F0027CE010E9472
:100A3000B400080F111D0C151D0511F7C801DF9139
:100A4000CF911F910F91FF90EF90DF90CF9008957D
:100A5000CF92DF92EF92FF920F931F93CF93DF938A
:100A6000E82FF0E0EE0FFF1FDF01A158BC4F8D9182
:100A70009C91DA01A823B923EF01C15ADC4FE88029
:100A8000F980CD018E0D9F1DE159FC4FC081D181B0
:100A9000AD01420F531FC417D50778F489016B01CC
:100AA000CA1BDB0BAE010E94D200A8014C1B5D0BE0
:100AB000B6016C0F7D1FC70101C0A901DF91CF9165
:100AC0001F910F91FF90EF90DF90CF900C94D20088
:100AD0008F929F92BF92CF92DF92EF92FF920F93ED
:100AE0001F93CF93DF9300D0CDB7DEB7B82E7A0136
:100AF00090E00496982E8824640184E2C80ED11CEC
:100B0000C60169837A830E94B400082F10E0102F79
:100B1000002785E2880E911CC4010E94B400080FD2
:100B2000111D9701A80169817A818B2D0E942805EA
:100B30000E0D1F1D612FC6010E949600602FC4017B
:100B40000F900F90DF91CF911F910F91FF90EF9039
:100B5000DF90CF90BF909F908F900C949600AF92B3
:100B6000BF92CF92DF92EF92FF920F931F93CF939A
:100B7000DF93DA01A901E82FF0E0EE0FFF1FEF018C
:100B8000C958DC4F888199816B01C822D922EF01B5
:100B9000C95ADC4FE880F980C6018E0D9F1DE959C6
:100BA000FC4FC081D1819601240F351FC217D30796
:100BB00080F48A015D01CC19DD09AE01BD010E94FE
:100BC000FA00A8014C1B5D0BB5016C0F7D1FC7011E
:100BD00001C0BD01DF91CF911F910F91FF90EF9068
:100BE000DF90CF90BF90AF900C94FA009F92AF929D
:100BF000BF92CF92DF92EF92FF920F931F93CF930A
:100C0000DF93982E6B017A01082F10E00C5F1F4FC5
:100C1000102F0027580188E2A80EB11CC5010E94C0
:100C2000B400C82FD0E0DC2FCC27075D1F4FC801D0
:100C30000E94B400C80FD11DDF93CF938BE691E0E3
:100C40009F938F930E948D0C9701A601BE01892D61
:100C50000E94AF05CE0DDF1D6D2FC5010E949600CD
:100C60000F900F900F900F906C2FC801DF91CF91D4
:100C70001F910F91FF90EF90DF90CF90BF90AF90BA
:100C80009F900C9496000F931F93CF93DF93C82FE0
:100C900083E891E00E94A30CD0E02496DC2FCC27BF
:100CA0008E010F5F1F4F60E1C8010E949600C801CE
:100CB0000E94B4008111FBCF6FEFCE010296DF914D
:100CC000CF911F910F910C949600CF92DF92EF92EB
:100CD000FF920F931F93CF93DF93C82FC62E8A01E5
:100CE000D22E8CE891E00E94A30C8FEF8C0DEC2E9D
:100CF000F12C8530D0F58C2F0E944306E701249615
:100D0000DC2FCC276C2D6D29CE010E949600CE01E0
:100D100004969E012B5F3F4F69010115110529F0D3
:100D2000612F0E949600602F0FC020918B0330919D
:100D30008C032F5F3F4F30938C0320938B03632FE3
:100D40000E94960060918B03C6010E9496008E015E
:100D50000F5F1F4F61E0C8010E949600C8010E940A
:100D6000B4008111FBCF11E001C010E0E70124962F
:100D7000DC2FCC27CE010E94B400082FCE010396B1
:100D80000E94B4001F920F931F928F9386E991E007
:100D90009F938F930E948D0C0F900F900F900F9048
:100DA0000F900F90812FDF91CF911F910F91FF90A6
:100DB000EF90DF90CF9008950F931F93CF93DF9321
:100DC000C82F87EB91E00E94A30CD0E02496DC2F83
:100DD000CC278E010D5F1F4FC8010E94B4008331E4
:100DE000D9F4219662E0CE010E949600CE010E94C5
:100DF000B4008111FBCFC8010E94B4001F928F93F1
:100E000081EC91E09F938F930E948D0C0F900F9037
:100E10000F900F9081E005C08FEC91E00E94A30C31
:100E200080E0DF91CF911F910F910895CF93DF93D1
:100E3000C82F86EE91E00E94A30CD0E0DC2FCC27D7
:100E4000CD5FDB4FCE010E94B4008431B1F4CE01FE
:100E50000E94B4008731D9F7CE010E94B4001F92DE
:100E60008F9381EC91E09F938F930E948D0C0F9054
:100E70000F900F900F9081E005C080EF91E00E94ED
:100E8000A30C80E0DF91CF910895EF92FF920F9332
:100E90001F93CF93DF93C82F8B017A0188E092E0F4
:100EA0000E94A30CF80160816F3F51F481818F3F54
:100EB00099F482818F3F81F483818F3F69F40FC061
:100EC00061110AC0F8018181811106C082818111FE
:100ED00003C08381882319F0E114F10431F48FEC0D
:100EE00091E00E94A30C80E02FC0D0E02496DC2F7C
:100EF000CC27CE010C960E949600F8016181CE01AC
:100F00000D960E949600F8016281CE010E960E9415
:100F10009600F8016381CE010F960E9496006F2D16
:100F2000CE0140960E9496006E2DCE0141960E9401
:100F30009600219664E0CE010E949600CE010E94A8
:100F4000B4008111FBCF81E0DF91CF911F910F9110
:100F5000FF90EF900895CF93DF93C82F85E092E044
:100F60000E94A30CD0E0DC2FCC27CF5FDB4F68E0E2
:100F7000CE010E949600CE010E94B4008111FBCFE9
:100F8000DF91CF9108958F929F92AF92BF92CF92AF
:100F9000DF92EF92FF921F93CF93DF93182F4B01B5
:100FA0007A0180E393E00E94A30C812F0E946900E4
:100FB0008E159F0520F4812F0E9469007C01C12FAE
:100FC000D0E02496DC2FCC275E0183E0A80EB11C74
:100FD000812F0E94B0046C01C5010E94B4008731CA
:100FE000A9F08C3199F0DF92CF921F921F9383E189
:100FF00092E09F938F930E948D0C0F900F900F9013
:101000000F900F900F90E12CF12C03C0CE14DF0451
:10101000F8F2A701B401812F0E9468056E018FEFDD
:10102000C81AD80A60E2C6010E949600C6010E9452
:10103000B4008111FBCF2296CE010E94B40084FD42
:101040000FC0C5010E94B4008111F6CF8BE392E07E
:101050000E94A30C812F0E94430680E090E005C00F
:1010600060E1CE010E949600C701DF91CF911F91F0
:10107000FF90EF90DF90CF90BF90AF909F908F90B8
:101080000895BF92CF92DF92EF92FF920F931F933A
:10109000CF93DF93B82E6B018A01C82FD0E024963E
:1010A000DC2FCC277E0183E0E80EF11CC7010E94F3
:1010B000B400873191F0C7010E94B4001F928F9352
:1010C00089E492E09F938F930E948D0C0F900F9074
:1010D0000F900F908FEF9FEF26C080E00E94EC04EE
:1010E0007C0118161906ECF48CE592E00E94A30C22
:1010F000E016F10620F00115110589F001C0870105
:10110000A801B6018B2D0E94F605219660E4CE0160
:101110000E949600CE010E94B4008111FBCFC8014D
:1011200002C080E090E0DF91CF911F910F91FF907E
:10113000EF90DF90CF90BF9008958F929F92BF92D3
:10114000CF92DF92EF92FF920F931F93CF93DF9393
:10115000B82E4B01EA01790184E692E00E94A30CCB
:101160008B2D0E9469008C179D0728F48B2D0E94FF
:1011700069006C0101C06E01F7016081611109C055
:101180008181811106C08281811103C083818823FE
:1011900031F00115110519F0C114D10429F5DF93BF
:1011A000CF931F930F93F70183811F928F938281B7
:1011B0001F928F9381811F928F931F926F931F9223
:1011C000BF928EE692E09F938F930E948D0C8FECDE
:1011D00091E00E94A30C8DB79EB740960FB6F8948D
:1011E0009EBF0FBE8DBF49C0CB2DD0E02496DC2F13
:1011F000CC27CE010C960E949600F7016181CE01AA
:101200000D960E949600F7016281CE010E960E9413
:101210009600F7016381CE010F960E949600612F20
:10122000CE0140960E949600602FCE0141960E940A
:101230009600A601B4018B2D0E9468058E010F5FF8
:101240001F4F60E2C8010E949600C8010E94B400CE
:101250008111FBCF2296CE010E94B40084FD10C004
:10126000CE010E94B40083FFF6CF8AE493E00E948F
:10127000A30C68E1CE010E94960080E090E005C0DA
:1012800060E1CE010E949600C601DF91CF911F91CF
:101290000F91FF90EF90DF90CF90BF909F908F9035
:1012A00008952F923F924F925F926F927F928F920A
:1012B0009F92AF92BF92CF92DF92EF92FF920F93E5
:1012C0001F93CF93DF93CDB7DEB72A970FB6F8946D
:1012D000DEBF0FBECDBF782E4B016A0179011A87A0
:1012E00009870E94EC04892B09F42BC186E992E05E
:1012F0000E94A30C872D0E94EC04682E392ECD2865
:1013000009F417C1472C512C84E0480E511C542C71
:101310004424520198E2A90EB11CC5010E94B400F8
:10132000082F10E0102F00276201E9E2CE0ED11C39
:10133000C6010E94B400080F111D3F926F921F93C7
:101340000F9382EA92E09F938F930E948D0CC201CB
:101350000E94B4000F900F900F900F900F900F907D
:101360008770833009F464C0843009F4ABC08230E4
:1013700009F0D0C028E030E0AE014F5F5F4FB80108
:10138000872D0E94AF051801F8E02F0E311C8981CE
:10139000F70180838A8181838B8182838C8183831F
:1013A0008D8190E0982F88272E81820F911DE985ED
:1013B000FA85918380830F8110E0102F00278885A4
:1013C000080F111D1F930F9382EC92E09F938F9350
:1013D0000E948D0CE985FA8581818F9380818F939E
:1013E00088ED92E09F938F930E948D0CF70183818B
:1013F0001F928F9382811F928F9381811F928F936F
:1014000080811F928F938BEE92E09F938F930E9427
:101410008D0C9801A401B101872D0E94AF057101C7
:10142000E00EF11E6F2DC5010E9496006E2D41C089
:1014300026E030E0AE014F5F5F4FB801872D0E947C
:10144000AF05180196E0290E311C8981F7018083D0
:101450008A8181838B8182838C8183830D8110E0DB
:10146000102F00278E81080F111D85E093E00E9448
:10147000A30CF70183811F928F9382811F928F9318
:1014800081811F928F9380811F928F938BEE92E0C8
:101490009F938F930E948D0C9801A401B101872D19
:1014A0000E94AF05200E311E632DC5010E949600DB
:1014B000622DC6010E9496000FB6F894DEBF0FBEE3
:1014C000CDBF2AC022E030E0AE014F5F5F4FB801D0
:1014D000872D0E94AF05780192E0E90EF11C098189
:1014E00010E0902F88270A8110E002501109080FA0
:1014F000191F9801A401B701872D0E94AF05E00EC6
:10150000F11E6F2DC5010E9496006E2DC6010E942E
:10151000960002C000E010E0EFEF4E1A5E0A60E4B1
:10152000C2010E949600C2010E94B4008111FBCF4B
:1015300002C000E010E089E193E00E94A30CC80122
:1015400002C080E090E02A960FB6F894DEBF0FBE8E
:10155000CDBFDF91CF911F910F91FF90EF90DF9062
:10156000CF90BF90AF909F908F907F906F905F9043
:101570004F903F902F900895CF92DF92FF920F935C
:101580001F93CF93DF93F82E6B01EA018CE293E077
:101590000E94A30C8F2D0E9469008C179D0728F4D0
:1015A0008F2D0E9469008C0101C08E01011511056B
:1015B00089F41F921F92DF93CF9388E393E09F9368
:1015C0008F930E948D0C0F900F900F900F900F90A3
:1015D0000F9030C0A801B6018F2D0E946805CF2D55
:1015E000D0E02496DC2FCC276E018FEFC81AD80AE2
:1015F00060E2C6010E949600C6010E94B4008111FB
:10160000FBCF6E0182E0C80ED11C2396C6010E945A
:10161000B40084FD12C0CE010E94B400C6010E9435
:10162000B40083FFF3CF86E493E00E94A30C8F2DD8
:101630000E94430680E090E005C060E1C6010E9480
:101640009600C801DF91CF911F910F91FF90DF901D
:10165000CF900895CF92DF92EF92FF920F931F9356
:10166000CF93DF936C017B018A01E9010E947F0225
:1016700065E585E50E942301C6010E94CE02C701EF
:101680000E94F102C8010E948202CE01DF91CF9137
:101690001F910F91FF90EF90DF90CF900C94B502C7
:1016A0008093BB0084E88093BC008091BC0087FFDE
:1016B000FCCF08951092B9008CE08093B80084E0CC
:1016C0008093BC000895CF9394EA9093BC009091CE
:1016D000BC0097FFFCCF9091B900987F983011F033
:1016E00080E015C0C62F880F0E94500B8091B90072
:1016F000887F8831A9F78C2F0E94500B8091B90008
:10170000887F883269F784E98093BC0081E0CF91BB
:101710000895CF93DF9394EA9093BC009091BC001E
:1017200097FFFCCF9091B900987F983011F080E03E
:101730001EC0C42FD62F880F0E94500B8091B90075
:10174000887F8831A1F78D2F0E94500B8091B900BE
:10175000887F883261F78C2F0E94500B8091B900EE
:10176000887F883221F784E98093BC0081E0DF9193
:10177000CF910895092E000CAA0BBB0B9C01AD0163
:1017800084E0220F331F441F551F8A95D1F760E074
:1017900074E284EF90E00E946B0C21503109309389
:1017A000C5002093C40088E18093C10086E0809347
:1017B000C200E0ECF0E080818D7F808308959091FD
:1017C000C00095FFFCCF8093C6000895CF93C82F2B
:1017D0008A3019F48DE00E94DF0B8C2F0E94DF0B02
:1017E00080E090E0CF9108958091C00087FFFCCF0A
:1017F0008091C600089580E895E20E94BA0B82E0CD
:1018000091E0909396038093950308950F931F930F
:10181000CF93DF93CDB7DEB764970FB6F894DEBFF2
:101820000FBECDBF86E0E0E1F1E0DE011196019050
:101830000D928A95E1F72CEA2F879AE1988B81E93E
:10184000898B3DEC3A8B2B879C878D878EEF8E871B
:101850008FEF8F83888789871A860E94FB0B9E01F2
:10186000295F3F4FAE01455F5F4FBE01615F7F4F14
:10187000CE0101960E942A0B20E044EE57E062E080
:10188000809156030E9465068823C1F020E044EE53
:1018900057E061E0809101010E946506882371F0A4
:1018A00001E913E02DE833E042E050E0BE016D5E57
:1018B0007F4F809156030E945109F2CF8FEF9FEF27
:1018C00064960FB6F894DEBF0FBECDBFDF91CF9107
:1018D0001F910F910895A1E21A2EAA1BBB1BFD01B7
:1018E0000DC0AA1FBB1FEE1FFF1FA217B307E407FF
:1018F000F50720F0A21BB30BE40BF50B661F771F57
:10190000881F991F1A9469F7609570958095909536
:101910009B01AC01BD01CF010895A0E0B0E0E3E977
:10192000FCE00C94610FAE014B5F5F4FFA016191D7
:101930007191AF0180919503909196030E94D30C11
:10194000E2E00C947D0F0F931F93CF93DF93E09110
:101950009503F0919603238121FF1BC08C01D0E0F9
:10196000C0E0F80181918F01609195037091960319
:10197000DB011896ED91FC911997882331F00995B8
:10198000892B79F3DFEFCFEFECCF8AE00995892B34
:1019900019F08FEF9FEF02C08D2F9C2FDF91CF9119
:1019A0001F910F910895ACE0B0E0E9EDFCE00C94DC
:1019B000510F7C016B018A01FC0117821682838121
:1019C00081FFBDC1CE0101964C01F7019381F60163
:1019D00093FD859193FF81916F01882309F4ABC139
:1019E000853239F493FD859193FF81916F018532A2
:1019F00029F4B70190E00E94BB0EE7CF512C312CA7
:101A000020E02032A0F48B3269F030F4803259F0BB
:101A1000833269F420612CC08D3239F0803339F47F
:101A2000216026C02260246023C0286021C027FDD9
:101A300027C030ED380F3A3078F426FF06C0FAE0C0
:101A40005F9E300D1124532E13C08AE0389E300D56
:101A50001124332E20620CC08E3221F426FD6BC17E
:101A6000206406C08C3611F4206802C0883641F428
:101A7000F60193FD859193FF81916F018111C1CF93
:101A8000982F9F7D9554933028F40C5F1F4FFFE3F0
:101A9000F9830DC0833631F0833771F0833509F057
:101AA0005BC022C0F801808189830E5F1F4F4424F0
:101AB0004394512C540115C03801F2E06F0E711C93
:101AC000F801A080B18026FF03C0652D70E002C040
:101AD0006FEF7FEFC5012C870E94B00E2C018301B0
:101AE0002C852F77222E17C03801F2E06F0E711C63
:101AF000F801A080B18026FF03C0652D70E002C010
:101B00006FEF7FEFC5012C870E94A50E2C012C855D
:101B10002068222E830123FC1BC0832D90E04816F1
:101B20005906B0F4B70180E290E00E94BB0E3A94EF
:101B3000F4CFF50127FC859127FE81915F01B70164
:101B400090E00E94BB0E31103A94F1E04F1A510818
:101B50004114510471F7E5C0843611F0893639F526
:101B6000F80127FF07C060817181828193810C5F3A
:101B70001F4F08C060817181072E000C880B990BE4
:101B80000E5F1F4F2F76722E97FF09C0909580959C
:101B9000709561957F4F8F4F9F4F2068722E2AE07E
:101BA00030E0A4010E94F30EA82EA81844C0853787
:101BB00029F42F7EB22E2AE030E025C0F22FF97FE3
:101BC000BF2E8F36C1F018F4883579F0B4C0803755
:101BD00019F0883721F0AFC02F2F2061B22EB4FE4C
:101BE0000DC08B2D8460B82E09C024FF0AC09F2F22
:101BF0009660B92E06C028E030E005C020E130E054
:101C000002C020E132E0F801B7FE07C060817181B7
:101C1000828193810C5F1F4F06C06081718180E0DB
:101C200090E00E5F1F4FA4010E94F30EA82EA8188B
:101C3000FB2DFF777F2E76FE0BC0372D3E7FA51440
:101C400050F474FE0AC072FC08C0372D3E7E05C0F9
:101C5000BA2C372D03C0BA2C01C0B52C34FF0DC0EF
:101C6000FE01EA0DF11D8081803311F4397E09C037
:101C700032FF06C0B394B39404C0832F867809F072
:101C8000B39433FD13C030FF06C05A2CB31418F4BC
:101C9000530C5B18B32CB31468F4B70180E290E0E6
:101CA0003C870E94BB0EB3943C85F5CFB31410F46F
:101CB0003B1801C0312C34FF12C0B70180E390E023
:101CC0003C870E94BB0E3C8532FF17C031FD03C02C
:101CD00088E790E002C088E590E0B7010CC0832F50
:101CE000867859F031FF02C08BE201C080E237FDF7
:101CF0008DE2B70190E00E94BB0EA51438F4B70145
:101D000080E390E00E94BB0E5A94F7CFAA94F401AE
:101D1000EA0DF11D8081B70190E00E94BB0EA11079
:101D2000F5CF332009F451CEB70180E290E00E9454
:101D3000BB0E3A94F6CFF7018681978102C08FEFF0
:101D40009FEF2C96E2E10C946D0FFC010590615021
:101D500070400110D8F7809590958E0F9F1F0895C1
:101D6000FC016150704001900110D8F7809590956A
:101D70008E0F9F1F08950F931F93CF93DF93FB0147
:101D8000238121FD03C08FEF9FEF28C022FF16C0E3
:101D900046815781248135814217530744F4A0813D
:101DA000B1819D012F5F3F4F318320838C9326812A
:101DB00037812F5F3F4F3783268310C0EB01092FF8
:101DC000182F0084F185E02D0995892BE1F68E818D
:101DD0009F8101969F838E83812F902FDF91CF91DA
:101DE0001F910F910895FA01AA27283051F120314F
:101DF00081F1E8946F936E7F6E5F7F4F8F4F9F4F9F
:101E0000AF4FB1E03ED0B4E03CD0670F781F891FE0
:101E10009A1FA11D680F791F8A1F911DA11D6A0FAE
:101E2000711D811D911DA11D20D009F468943F9161
:101E30002AE0269F11243019305D3193DEF6CF0160
:101E40000895462F4770405D4193B3E00FD0C9F726
:101E5000F6CF462F4F70405D4A3318F0495D31FD93
:101E60004052419302D0A9F7EACFB4E0A6959795E6
:101E7000879577956795BA95C9F7009761057105BC
:101E800008959B01AC010A2E069457954795379506
:101E90002795BA95C9F7620F731F841F951FA01D60
:101EA00008952F923F924F925F926F927F928F92FE
:101EB0009F92AF92BF92CF92DF92EF92FF920F93D9
:101EC0001F93CF93DF93CDB7DEB7CA1BDB0B0FB6E3
:101ED000F894DEBF0FBECDBF09942A8839884888A0
:101EE0005F846E847D848C849B84AA84B984C88436
:101EF000DF80EE80FD800C811B81AA81B981CE0F2D
:101F0000D11D0FB6F894DEBF0FBECDBFED01089511
:041F1000F894FFCF73
:101F140001010000000200000000E60B00000000C8
:101F2400A0BDCDDDEDFD737973696E697428290D4B
:101F3400004368616E6E656C203A2053454E442020
:101F44004D454D2053495A45203A20524543562089
:101F54004D454D2053495A450D002564203A20250E
:101F64002E3478203A20252E3478203A20252E3419
:101F740078203A20252E34780D0A004953525F52B6
:101F8400583A2072645F707472203A20252E347897
:101F94000D0A00636C6F736528290D00736F636B02
:101FA400657428290D00536E5F5352203D20252E61
:101FB4003278202C2050726F746F636F6C203D2038
:101FC400252E32780D0A006C697374656E28290D0C
:101FD40000737461747573203D2025780D0A0046E2
:101FE40061696C5B696E76616C69642069702C70E0
:101FF4006F72745D0D0061636365707428290D0050
:102004004661696C5B6E6F74206C697374656E698C
:102014006E675D0D00646973636F6E6E656374282B
:10202400290D00736F636B657420256420667265E7
:102034006573697A652825642920656D7074792033
:102044006F72206572726F720D0A00534F434B5FBB
:10205400434C4F5345442E0D004261642073746118
:10206400747573203D20253032780A0072656376DA
:1020740028290D0073656E64746F28290D0025648A
:10208400204661696C5B252E32782E252E32782EFF
:10209400252E32782E252E32782C20252E642C20C5
:1020A40025645D0D0A007265637666726F6D28297A
:1020B4000D004953525F52583A2072645F70747233
:1020C400203A20252E34782073697A653D25640DE5
:1020D4000A00554450206D736720232564206172E3
:1020E40072697665640D0A00736F757263652050BA
:1020F4006F7274203A2025750D0A00736F75726330
:1021040065204950203A2025642E25642E25642E0E
:1021140025640D0A00495020524157206D736720F1
:10212400617272697665640D007265637666726FBA
:102134006D282920656E64202E2E0D0069676D7050
:1021440073656E6428290D002564204661696C5B03
:1021540025645D0D0A0069676D7073656E642066A1
:0621640061696C2E0D0004
:00000001FF
